:1000000019C033C032C031C030C02FC02EC02DC087
:100010002CC02BC02AC081C028C027C026C025C044
:1000200024C023C022C021C020C01FC01EC01DC0CC
:100030001CC01BC011241FBECFEFD4E0DEBFCDBF5C
:1000400011E0A0E0B1E0E0E0F9E002C005900D921F
:10005000A432B107D9F721E0A4E2B1E001C01D92BA
:10006000AC32B207E1F71DD349C4CACF8FEF8AB9CA
:1000700087E084B980E388B93B9843981092800068
:100080008AE08093810084EC99E0909389008093CA
:100090008800EFE6F0E080818260808378940895A4
:1000A0009DEC899F912D1124969596959695E0E06B
:1000B000F1E09283990F292F220F220F920F891BB3
:1000C000818360830895349906C080912B018F5FEE
:1000D00080932B0102C010922B0135990AC08091A8
:1000E0002A018F5F80932A0190912B01933368F04E
:1000F00006C010922A0180912B01833368F0109280
:100100002B0181E0809329010895833328F0109218
:100110002A0182E08093290108951F920F920FB661
:100120000F9211242F933F934F935F936F937F937D
:100130008F939F93AF93BF93EF93FF9315B81BB823
:100140008DE08A95F1F7000081E090E000902401B5
:1001500002C0880F991F0A94E2F785B9E091240143
:10016000F0E0E050FF4FE081F0E0ED5FFE4F808176
:100170008BB9809124018F5F833018F48093240120
:1001800002C0109224019FDFFF91EF91BF91AF91C8
:100190009F918F917F916F915F914F913F912F919F
:1001A0000F900FBE0F901F901895E0E0F1E090E1E6
:1001B0009283918390832FEB35E444E021503040CB
:1001C0004040E1F700C00000813021F0823009F4A6
:1001D000E2C0C1C1E0E0F1E022E1228390E191833D
:1001E00090835FEB65E474E0515060407040E1F74C
:1001F00000C000003CE03283918390838FEBA5E444
:1002000044E08150A0404040E1F700C0000088E099
:100210008283918390835FEB65E474E0515060408A
:100220007040E1F700C00000828321839083AFEB30
:1002300045E454E0A15040405040E1F700C00000C8
:100240008283318390836FEB75E4A4E0615070404A
:10025000A040E1F700C000008283818390834FEBD0
:1002600055E464E0415050406040E1F700C00000B8
:100270008283818341E040837FEBA5E454E07150A9
:10028000A0405040E1F700C000008283818353E02A
:1002900050836FEB75E4A4E061507040A040E1F73B
:1002A00000C000008283818380836FEB75E4A4E04B
:1002B00061507040A040E1F700C00000828381835C
:1002C00080836FEB75E4A4E061507040A040E1F7DB
:1002D00000C000008283818350835FEB65E474E09B
:1002E000515060407040E1F700C00000828381837C
:1002F0004083AFEB45E454E0A15040405040E1F76B
:1003000000C000008283818390836FEB75E4A4E0DA
:1003100061507040A040E1F700C00000828331834B
:1003200090834FEB55E464E0415050406040E1F76A
:1003300000C000008283218390837FEBA5E444E02A
:100340007150A0404040E1F700C0000082839183DB
:1003500090835FEB65E474E0515060407040E1F7DA
:1003600000C000003283918390838FEBA5E434E0DA
:100370008150A0403040E1F700C00000228391830B
:1003800090834FEB55E464E0415050406040E1F70A
:1003900000C00000E0C0E0E0F1E022E1228380E163
:1003A000818380837FEB95E4A4E071509040A0406E
:1003B000E1F700C000003CE03283818380834FEB93
:1003C00055E464E0415050406040E1F700C0000057
:1003D00098E09283818380837FEBA5E444E07150B1
:1003E000A0404040E1F700C0000092832183808359
:1003F0005FEB65E474E0515060407040E1F700C08D
:100400000000928331838083AFEB45E454E0A15038
:1004100040405040E1F700C0000092839183808308
:100420006FEB75E4A4E061507040A040E1F700C0BC
:1004300000009283918341E040835FEB65E474E0C8
:10044000515060407040E1F700C0000092839183FA
:1004500053E05083AFEB65E474E0A150604070401E
:10046000E1F700C00000928391839083AFEB65E4D5
:1004700074E0A15060407040E1F700C0000052837A
:1004800091839083AFEB65E474E0A15060407040CD
:10049000E1F700C00000428391839083AFEB65E4F5
:1004A00074E0A15060407040E1F700C0000082831A
:1004B00091839083AFEB65E474E0A150604070409D
:1004C000E1F700C00000828351839083AFEB55E4D5
:1004D00064E0A15050406040E1F700C0000082831A
:1004E000418390837FEBA5E444E07150A0404040FD
:1004F000E1F700C000008283818390835FEB65E4B5
:1005000074E0515060407040E1F700C00000828309
:10051000818330839FEBA5E434E09150A0403040CC
:10052000E1F700C000008283818320834FEB55E414
:1005300064E0415050406040E1F700C00000828319
:10054000818380837FEB85E494E07150804090400C
:10055000E1F700C00000E0E0F1E080E18283818308
:100560008083AFEB25E434E0A15020403040E1F738
:1005700000C0000008950F931F93CF93DF9300D026
:1005800000D01F92CDB7DEB73B9889EC07C036E0AC
:100590003A95F1F700C0815009F46EC03399F7CF56
:1005A00086E507C096E09A95F1F700C0815009F4FE
:1005B00065C0339BF7CF86E507C0A6E0AA95F1F7A3
:1005C00000C0815009F45CC03399F7CFFE01319629
:1005D00085E0DF011D928A95E9F7AE014A5F5F4F22
:1005E00022C0B6E0BA95F1F700C0915011F44AC0AC
:1005F00098E3339BF6CF38EC3A95F1F7220F339915
:1006000008C00BC0A6E0AA95F1F700C0915011F404
:100610003BC09EE23399F6CF2160815049F7219388
:100620004E175F0719F088E020E0E2CFA981B0E023
:10063000EA81F0E06B8170E04C8150E09D012E0F6B
:100640003F1F260F371F240F351F33270D8110E062
:1006500020173107D9F4BA2FAA27EA0FFB1FF0930E
:100660002801E0932701762F6627460F571F5093E6
:100670002601409325010BC082E009C083E007C03A
:1006800084E005C085E003C086E001C087E00F90EC
:100690000F900F900F900F90DF91CF911F910F91BE
:1006A0000895E4DCE0E0F1E090E1928391839083AF
:1006B000AFE4B3EC1197F1F700C0000083E182834F
:1006C00091839083BFE70FE412E1B15000401040E6
:1006D000E1F700C000008283818390832FE73FE42D
:1006E00042E1215030404040E1F700C000008283E9
:1006F000818380838FE79FE4A2E181509040A040F6
:10070000E1F700C0000035E080E123E1D9E1C7E076
:10071000BAE196E1ABE17CE16DE15EE182832183A8
:10072000D0830FEB15E444E0015010404040E1F766
:1007300000C0000082838183C0830FEB15E444E096
:10074000015010404040E1F700C0000082838183E7
:10075000B0830FEB15E444E0015010404040E1F756
:1007600000C0000082839183A0830FEB15E444E076
:10077000015010404040E1F700C000009283918397
:1007800090830FEB15E444E0015010404040E1F746
:1007900000C000007283918380830FEB15E444E076
:1007A000015010404040E1F700C0000062838183A7
:1007B00080830FEB15E444E0015010404040E1F726
:1007C00000C000005283818380830FEB15E444E076
:1007D000015010404040E1F700C000000FE10283EB
:1007E000218380831FEB45E404E01150404000402A
:1007F000E1F700C000002283218320831FEB45E442
:1008000004E0115040400040E1F700C000003150CA
:1008100009F084CFE0E0F1E080E18283818380838E
:100820001FEF2EE934E2115020403040E1F700C0C4
:100830000000EF010CE010E1809129018130B1F15D
:1008400020F0823009F440C0F9CF339B25C03B9A99
:1008500043984FE788E391E0415080409040E1F7B2
:1008600000C0000088DE811110C020912701309166
:100870002801ADECBCEC36D096958795969587957A
:10088000969587956FE00CDC03C00A8389831883F3
:10089000809129018111D0CFAFE7B4E82EE1A150BA
:1008A000B0402040E1F700C00000C6CF81E07DDC11
:1008B000109229013FEF44E38CE0315040408040EA
:1008C000E1F700C00000B8CF82E06FDC1092290190
:1008D0009FEFA4E3BCE09150A040B040E1F700C01E
:1008E0000000AACFA29FB001B39FC001A39F01D077
:1008F000B29F700D811D1124911D0895F894FFCFB2
:10090000101010FC24BAAE66CEDEA4FEEE161EDA7F
:1009100012ADF3000250802004081040A02C0C18E7
:0409200058D0C000EB
:00000001FF
